:0200000480007A
:100000006F00C004732F2034930F8000630AFF0336
:10001000930F90006306FF03930FB0006302FF038A
:10002000170F0080130F0FFE63040F0067000F000F
:10003000732F203463540F006F004000136E9E53E3
:10004000171F00002320CFFD6FF09FFF732540F1A5
:100050006310050073251030635805000F00F00F82
:10006000130E100073000000130E00009702000032
:10007000938282F973905230735020307350303035
:1000800073504030970200809382C2F7638C020065
:10009000739052109302B01A739022307323203061
:1000A000E39E62F873500030970200009382420191
:1000B00073901234732540F17300203097200000B4
:1000C000938040F43701AA001301A10A23A0200065
:1000D00083A10000B70EAA00938EAE0A130E200073
:1000E0006390D147972000009380C0F137B100AAF8
:1000F000130101A023A2200083A14000B7BE00AAE3
:10010000938E0EA0130E3000639CD1439720000005
:10011000938040EF3711A00A130101AA23A4200005
:1001200083A18000B71EA00A938E0EAA130E400072
:100130006398D141972000009380C0EC37A10AA0BA
:100140001301A10023A6200083A1C000B7AE0AA01E
:10015000938EAE00130E50006394D13F97200000A1
:10016000938000EC3701AA001301A10A23AA20FE04
:1001700083A140FFB70EAA00938EAE0A130E600053
:100180006390D13D97200000938080E937B100AAA9
:10019000130101A023AC20FE83A180FFB7BE00AAFB
:1001A000938E0EA0130E7000639CD139972000002F
:1001B000938000E73711A00A130101AA23AE20FEA5
:1001C00083A1C0FFB71EA00A938E0EAA130E800053
:1001D0006398D13797200000938080E437A10AA06C
:1001E0001301A10023A0200083A10000B7AE0AA044
:1001F000938EAE00130E90006394D13597200000CB
:10020000938040E23751341213018167138200FE5C
:100210002320220283A10000B75E3412938E8E67E2
:10022000130EA000639ED13197200000938080DFE1
:1002300037312158130181099380D0FFA3A32000F7
:1002400017220000130242DE83210200B73E21582C
:10025000938E8E09130EB0006394D12F130EC0003D
:1002600013020000B7D0BBAA9380D0CD17210000A5
:10027000130141D92320110083210100B7DEBBAA5D
:10028000938EDECD639ED12B1302120093022000C9
:10029000E31A52FC130ED00013020000B7C0ABDA11
:1002A0009380D0CC172100001301C1D513000000AA
:1002B0002322110083214100B7CEABDA938EDECC2E
:1002C0006390D1291302120093022000E31852FC1C
:1002D000130EE00013020000B7C0AADD9380C0BC7B
:1002E00017210000130101D21300000013000000C9
:1002F0002324110083218100B7CEAADD938ECEBCCA
:100300006390D1251302120093022000E31652FCE1
:10031000130EF00013020000B7B0DACD9380C0BB1B
:1003200013000000172100001301C1CD2326110086
:100330008321C100B7BEDACD938ECEBB6392D121AB
:100340001302120093022000E31852FC130E000166
:1003500013020000B7B0DDCC9380B0AB13000000F7
:1003600017210000130101CA130000002328110007
:1003700083210101B7BEDDCC938EBEAB6392D11D4C
:100380001302120093022000E31652FC130E100118
:1003900013020000B7E0CDBC9380B0AA13000000A8
:1003A00013000000172100001301C1C5232A11000A
:1003B00083214101B7EECDBC938EBEAA6392D119C1
:1003C0001302120093022000E31652FC130E2001C8
:1003D00013020000172100001301C1C2B720110051
:1003E000938030232320110083210100B72E1100B8
:1003F000938E3E236396D1151302120093022000C0
:10040000E31A52FC130E3001130200001721000002
:10041000130141BFB7100130938030221300000058
:100420002322110083214100B71E0130938E3E220A
:100430006398D1111302120093022000E31852FCBA
:10044000130E40011302000017210000130181BBAD
:10045000B710003393802012130000001300000037
:100460002324110083218100B71E0033938E2E12A6
:100470006398D10D1302120093022000E31652FC80
:10048000130E50011302000017210000130181B761
:1004900013000000B70030239380201123261100A1
:1004A0008321C100B70E3023938E2E11639AD10998
:1004B0001302120093022000E31852FC130E600195
:1004C00013020000172100001301C1B31300000044
:1004D000B70033229380100113000000232811007D
:1004E00083210101B70E3322938E1E01639AD10539
:1004F0001302120093022000E31652FC130E700147
:1005000013020000172100001301C1AF1300000007
:1005100013000000B730231293801000232A11002B
:1005200083214101B73E2312938E1E00639AD101AD
:100530001302120093022000E31652FC631CC00158
:100540000F00F00F63000E00131E1E00136E1E003E
:10055000730000000F00F00F130E10007300000076
:10056000731000C000000000000000000000000048
:10057000000000000000000000000000000000007B
:040580000000000077
:1010000000000000000000000000000000000000E0
:1010100000000000000000000000000000000000D0
:1010200000000000000000000000000000000000C0
:1010300000000000000000000000000000000000B0
:081040000000000000000000A8
:10200000EFBEADDEEFBEADDEEFBEADDEEFBEADDEF0
:10201000EFBEADDEEFBEADDEEFBEADDEEFBEADDEE0
:10202000EFBEADDEEFBEADDE000000000000000040
:040000058000200057
:00000001FF
